:100000000C94B0070C94F7070C94F7070C94F707BF
:100010000C94F7070C94F7070C94F7070C94F70768
:100020000C94F7070C94F7070C947E130C9450145F
:100030000C94F7070C94F7070C94F7070C94F70748
:100040000C94F7070C94142D0C94F7070C94F707F5
:100050000C94F7070C940D230C94F7070C94F707F6
:100060000C94F7070C94F7070C94F7070C94F70718
:100070000C94F7070C94F7070C94F7070C94F70708
:100080000C94F7070C94F7070C94F7070C94F707F8
:100090000C94F7070C94F7070C94F7070C94F707E8
:1000A0000C94F7070C94F7070C94F707BD14DF14B2
:1000B000D215DF14D21524154715D2159C15AF158E
:1000C000FD18FD182C192C196F19A919B61BB61B90
:1000D000C219B61BB71AB71A8A1BB61BB61BA11BCF
:1000E00000F001F002F0F0A3F0A42B00340039007E
:1000F000E100E00000001E00140004001D00E2000A
:10010000007F1F001A0016001B0003522800200069
:10011000080007000600E3002C002100150009007C
:10012000190064002D00220017000A0005000000DD
:1001300050002E004A0000000154000052002E0022
:100140004D00000002540000510023001C000B0071
:10015000110000004F00240018000D001000E60000
:100160002D0025000C000E003600E7002C002600B4
:1001700012000F003700035228002700130033003D
:100180003800E60000772A002F003100E500E40087
:1001900000002B0006003900E100E00000001E0016
:1001A000130007003400E200007F1F0017000B005F
:1001B0001400035228002000090033001500E3005A
:1001C0002C0021000E0012001A0004522D00220003
:1001D0000F000C001100000050002E004A0000002B
:1001E0000100000052002E004D0000000100000040
:1001F00051002300050018000D0000004F002400EE
:1002000004003800100004522D00250016001C00C8
:100210003600E7002C0026000A00080037000352D1
:100220002800270019001B002D00E60000772A0097
:100230001D003100E500E40000002B001D0000005F
:10024000E100E00000001E001B0018002F00E2008B
:10025000007F1F0019000C0033000352280020000B
:100260000F0004003400E3002C0021000600080009
:10027000130004522D0022001A0012001C0000007E
:1002800050002E004A0000000100000052002E0025
:100290004D00000001000000510023000E00160078
:1002A000050000004F0024000B0011001000045254
:1002B0002D0025000A0015003600E7002C0026005E
:1002C0000900170037000352280027001400070018
:1002D0000D00E60000772A002D000000E500E40094
:1002E0000000010001000100010001000000010008
:1002F00001000100010001000100010001000100F6
:1003000001000100010001000100010001000100E5
:100310000100010013A715A701000100F40001006E
:100320000100010001000000F200010001000000D6
:1003300001000000F00001000100000001000000C9
:10034000F10001000100010001000000F3000100C4
:1003500042003E003A000100F500010043003F006A
:100360003B00010001000100440040003C0001008E
:1003700001000100450041003D00010001000100B5
:100380000100010001000100000000000000000069
:1003900000000000000000004B004A00290000009F
:1003A000000000002A0050002B00010000000000A7
:1003B0005200510049000000000000004C004F00B6
:1003C00028000100000000004E004D007A000000EF
:1003D000000000000000000001000000000000001C
:1003E000000000000100000000000000000000000C
:1003F0000000000000000000240021001E00010099
:1004000000000000250022001F0000000000000086
:10041000260023002000010000000000300036000C
:10042000000000000000000038003700000000005D
:1004300000000A002530313662003A2000253032B3
:1004400058000A722F632030313233343536373852
:10045000394142434445460A000A002530325800DB
:10046000626F756E6365213A20006C656674207357
:100470006964652061747461636865640A006C6511
:1004800066742073696465206E6F74207265737082
:100490006F6E64696E670A00747279696E672074A2
:1004A0006F207265736574206D637032333031383C
:1004B0000A000A44454255473A20656E61626C6500
:1004C000642E0A005B735D004B6579626F61726434
:1004D0002073746172742E0A005B575D005B535D7C
:1004E000005B525D005B445D005B435D00160345AD
:1004F00000720067006F0044006F00780020004524
:10050000005A00000016034500720067006F0044A7
:10051000006F007800200045005A00000004030925
:100520000409028D00050100A0FA0904000001037E
:10053000010100092111010001223F00070581038B
:1005400008000A0904010001030102000921110148
:100550000001224D000705820308000A0904020079
:1005600001030000000921110100012236000705E6
:10057000830308000A0904030002030000000921A4
:100580001101000122200007058403200001070556
:1005900004032000010904040001030000000921F4
:1005A0001101000122390007058503100001120125
:1005B000100100000008EDFE071301000102000118
:1005C00005010906A101050719E029E71500250124
:1005D0009508750181020508190129059505750120
:1005E00091029501750391010507190029771500FE
:1005F0002501957875018102C00631FF0974A101BA
:100600000975150025FF95207508810209761500EA
:1006100025FF952075089102C005010980A101857B
:100620000216010026B7001A01002AB700751095BE
:10063000018100C0050C0901A101850316010026F6
:100640009C021A01002A9C02751095018100C005C8
:10065000010902A1010901A10005091901290515D6
:10066000002501950575018102950175038101053C
:1006700001093009311581257F9502750881060928
:10068000381581257F950175088106050C0A380209
:100690001581257F950175088106C0C005010906F1
:1006A000A101050719E029E7150025019508750145
:1006B0008102950175088101050819012905950533
:1006C000750191029501750391010507190029FF34
:1006D000150025FF950675088100C00A00253032F7
:1006E0005820006B6579626F6172645F7265706F2C
:1006F00072743A20000A0025303258006B65796226
:100700006F6172645F7365745F6C65643A20006446
:10071000656C5F6B65795F6269743A2063616E270F
:10072000742064656C3A20253032580A0061646494
:100730005F6B65795F6269743A2063616E2774202C
:100740006164643A20253032580A00646F6E652E69
:100750000A00626F6F676D61676963207363616E22
:100760003A202E2E2E2000290A002575002F002564
:1007700075005D2800256400200025640020002508
:10078000640020002564007C0025303258006D6F25
:100790007573656B6579205B62746E7C7820792057
:1007A0007620685D287265702F61636C293A205B42
:1007B000006D6B5F776865656C5F74696D655F740C
:1007C0006F5F6D6178203D2025640A006D6B5F7757
:1007D0006865656C5F6D61785F7370656564203D09
:1007E0002025640A006D6B5F74696D655F746F5FCF
:1007F0006D6178203D2025640A006D6B5F6D617826
:100800005F7370656564203D2025640A006D6B5F31
:10081000696E74657276616C203D2025640A006DF6
:100820006B5F64656C6179203D2025640A006D6B07
:100830005F776865656C5F74696D655F746F5F6D28
:100840006178203D2025640A006D6B5F77686565DF
:100850006C5F6D61785F7370656564203D20256411
:100860000A006D6B5F74696D655F746F5F6D6178B1
:10087000203D2025640A006D6B5F6D61785F7370A9
:10088000656564203D2025640A006D6B5F696E74A8
:10089000657276616C203D2025640A006D6B5F6493
:1008A000656C6179203D2025640A000A00257500E9
:1008B000363A20776865656C5F74696D655F746F43
:1008C0005F6D61783A20000A00257500353A20777F
:1008D0006865656C5F6D61785F73706565643A200B
:1008E000000A00257500343A2074696D655F746FE5
:1008F0005F6D61783A20000A00257500333A206D5B
:1009000061785F73706565643A20000A00257500A0
:10091000323A20696E74657276616C286D73293A7B
:1009200020000A00257500313A2064656C61792841
:100930002A31306D73293A20000A092D2056616C46
:10094000756573202D0A004D3E004D25643E200044
:100950003F007365742064656661756C740A0043BA
:100960003E200077686572652064656C74613A208A
:10097000637572736F723D25642C20776865656CB2
:100980003D25640A53656520687474703A2F2F659D
:100990006E2E77696B6970656469612E6F72672F5F
:1009A00077696B692F4D6F7573655F6B6579730A36
:1009B000000A092D204D6F7573656B6579202D0A2E
:1009C0004553432F713A09717569740A313A0964C4
:1009D000656C6179282A31306D73290A323A0969C8
:1009E0006E74657276616C286D73290A333A096DED
:1009F00061785F73706565640A343A0974696D657E
:100A00005F746F5F6D61780A353A09776865656C68
:100A10005F6D61785F73706565640A363A0977685F
:100A200065656C5F74696D655F746F5F6D61780A91
:100A30000A703A097072696E742076616C7565731C
:100A40000A643A097365742064656661756C747331
:100A50000A75703A092B310A646F776E3A092D31A5
:100A60000A706775703A092B31300A7067646F77C6
:100A70006E3A092D31300A0A7370656564203D2095
:100A800064656C7461202A206D61785F73706565A0
:100A900064202A2028726570656174202F20746993
:100AA0006D655F746F5F6D6178290A003F004D3E90
:100AB0002000433E20004C25640A000A092D2043F3
:100AC0006F6E736F6C65202D0A4553432F713A0981
:100AD000717569740A6D3A096D6F7573656B657927
:100AE0000A000A092D204D61676963202D0A643AC6
:100AF0000964656275670A783A09646562756720FA
:100B00006D61747269780A6B3A0964656275672071
:100B10006B6579626F6172640A6D3A09646562752A
:100B200067206D6F7573650A763A09766572736929
:100B30006F6E0A733A097374617475730A633A09C4
:100B4000636F6E736F6C65206D6F64650A302D3452
:100B50003A096C61796572302D34284631302D4662
:100B600034290A506175733A09626F6F746C6F6152
:100B70006465720A653A09656570726F6D0A6E3A4E
:100B8000094E4B524F0A7A3A09736C656570204CD6
:100B9000454420746573740A000A002575002E6EA2
:100BA0006B726F3A20000A002575002E7377617012
:100BB0005F6261636B736C6173685F6261636B73C7
:100BC000706163653A20000A002575002E73776115
:100BD000705F67726176655F6573633A20000A0033
:100BE0002575002E6E6F5F6775693A20000A002533
:100BF00075002E737761705F72616C745F726775D8
:100C0000693A20000A002575002E737761705F6CC9
:100C1000616C745F6C6775693A20000A0025750085
:100C20002E636170736C6F636B5F746F5F636F6E65
:100C300074726F6C3A20000A002575002E7377617C
:100C4000705F636F6E74726F6C5F636170736C6FF3
:100C5000636B3A20000A0025303258006B65796DCD
:100C600061705F636F6E6669672E7261773A20000C
:100C70000A002575002E6D6F7573653A20000A0015
:100C80002575002E6B6579626F6172643A20000AE7
:100C9000002575002E6D61747269783A20000A0093
:100CA0002575002E656E61626C653A20000A00258C
:100CB0003032580064656275675F636F6E6669679E
:100CC0002E7261773A20000A00257500646566611E
:100CD000756C745F6C617965723A20003F004E4B11
:100CE000524F3A206F66660A004E4B524F3A206FC1
:100CF0006E0A0074696D65725F636F756E743A2079
:100D00002530346C580A006B6579626F6172645FDC
:100D10006E6B726F3A2025580A006B6579626F61BD
:100D200072645F69646C653A2025580A006B6579C6
:100D3000626F6172645F70726F746F636F6C3A2080
:100D400025580A00686F73745F6B6579626F617212
:100D5000645F6C65647328293A2025580A000A09E3
:100D60002D20537461747573202D0A004743433A54
:100D700020352E332E30204156522D4C4942433AD5
:100D800020312E382E3173766E204156525F4152FB
:100D900043483A20617672350A004F5054494F4E0D
:100DA000533A204C55464120424F4F544D414749FC
:100DB00043204D4F5553454B4559204558545241BA
:100DC0004B455920434F4E534F4C4520434F4D4DBB
:100DD000414E44204E4B524F203531320A0042558D
:100DE000494C443A20323030363038342D64697200
:100DF0007479202831313A35303A3438204A616EDE
:100E00002033302032303136290A005649443A2006
:100E1000307846454544284572676F446F782045D1
:100E20005A29205049443A20307831333037284508
:100E300072676F446F7820455A29205645523A20F0
:100E40003078303030310A00444553433A20742E14
:100E50006D2E6B2E206B6579626F617264206669FE
:100E6000726D7761726520666F72204572676F647C
:100E70006F780A000A092D2056657273696F6E201B
:100E80002D0A000A6D6F7573653A206F66660A0059
:100E90000A6D6F7573653A206F6E0A000A6B65798B
:100EA000626F6172643A206F66660A000A6B657948
:100EB000626F6172643A206F6E0A000A6D6174722B
:100EC00069783A206F66660A000A6D617472697803
:100ED0003A206F6E0A000A64656275673A206F6E89
:100EE0000A000A64656275673A206F66660A000A3E
:100EF0000A626F6F746C6F616465722E2E2E200013
:100F0000433E20006565636F6E6669673A0A005369
:100F10006C656570204C454420746573740A00004C
:100F200000000000000000000000010204060A0F9B
:100F300017202C3A4A5D71879DB3C7DAE9F5FCFFAB
:100F4000FCF5E9DAC7B39D87715D4A3A2C20170F8B
:100F50000A0604020100000000000000000000007A
:100F600011241FBECFEFDAE0DEBFCDBF04B603FE13
:100F700027C08091F8019091F901A091FA01B091F8
:100F8000FB018730904BA740B04BD1F41092F80191
:100F90001092F9011092FA011092FB0114BE84B76D
:100FA000877F84BF0FB6F894A89580916000886110
:100FB00080936000109260000FBEE0E0FFE30995AF
:100FC00011E0A0E0B1E0E2EEFDE502C005900D9277
:100FD000AA33B107D9F721E0AAE3B1E001C01D921D
:100FE000A83FB207E1F70E94B9100C94EF2E0C94C1
:100FF0000000FF93EF93E0913A01F0913B013097AD
:1010000009F00995EF91FF910895FC0185918030D9
:1010100011F0EFDFFBCF0895FF27E0E230E247FF5A
:101020000CC0419597FF09C0EDE2609570958095E1
:101030009095611D711D811D911D27FF02C0219595
:1010400030E350E2AA27660F771F881F991FAA1F57
:10105000A41710F0A41B63955A95A9F7AA3008F0BD
:10106000A95FA05DAF93F3956115710581059105A9
:1010700041F7ED3211F4EF93F395F21718F43F9323
:10108000F395FBCF8F91B5DFFA95E1F70895E991DC
:10109000F9918591803021F0853219F0AADFF9CFDE
:1010A000089520E0E89455915532C1F3503311F47E
:1010B000689455915A3348F4505390F3220F022EFE
:1010C000220F220F200D250FF4CF0EF421958991C8
:1010D0009991533619F3533729F1533559F1BC011E
:1010E00088279927E8945C3621F48991999168942E
:1010F0005591543639F446EF7EF077FF0DC08FEFEF
:101100009FEF0AC055374AE039F0583540E121F0E9
:10111000523642E009F00895FF93EF937DDFEF919F
:10112000FF91B7CFFF93EF93FC0181918030B9F32A
:1011300060DFFBCFFF93EF9368DFF1CFDF93CF93B7
:10114000CDB7DEB72596A3DFCF91DF91089561116A
:101150000BC0FC018281882321F085EE0E94971745
:1011600003C085EE0E945F1880E090E00895089526
:101170006091BC017091BD018091BE019091BF0151
:101180000E940E2256985E9825982D9826982E98A3
:1011900027982F98823051F0833029F0813049F41C
:1011A000269A2E9A0895259A2D9A0895279A2F9A6D
:1011B000089556985E98089588EB98E0892B11F071
:1011C0000E94B80880E090E0089556985E982598AF
:1011D0002D9826982E9827982F988FEF90E090932F
:1011E00089008093880090938B0080938A0090936D
:1011F0008D0080938C00259A2D9A2FEF80E792E046
:10120000215080409040E1F700C00000269A2E9ABD
:101210002FEF80E792E0215080409040E1F700C03E
:101220000000279A2F9A2FEF80E792E0215080400C
:101230009040E1F700C0000025982D982FEF80E73F
:1012400092E0215080409040E1F700C000002698D5
:101250002E982FEF80E792E0215080409040E1F7F8
:1012600000C0000027982F9856985E9825982D98D2
:1012700026982E9827982F98089589EA80938000C1
:1012800089E08093810024982C983F988AB18F74CC
:101290008AB96E98479A8BB1806B8BB9769A0E9407
:1012A000E50887EB98E0892B11F00E94B70880E0F1
:1012B00090E0089580E28093000180913C018111CB
:1012C0000EC00E94A90981E080933C012FEF83EDBD
:1012D00090E3215080409040E1F700C0000080E49E
:1012E0000E94AF098093000181112EC00E94D9098C
:1012F00080930001811128C00E94D90980930001C8
:10130000811122C08FE30E94D909809300018111CD
:101310001BC00E94D10980E40E94AF0980930001A4
:10132000811112C08CE00E94D909809300018111C3
:101330000BC00E94D90980930001811105C08FE381
:101340000E94D909809300010E94D1098091000177
:1013500008951092B9008AE08093B800089594EA45
:101360009093BC009091BC0097FFFCCF9091B90086
:10137000987F983021F0903111F081E008958093AA
:10138000BB0084E88093BC008091BC0087FFFCCF49
:101390008091B900887F883111F0803471F780E046
:1013A000089584E98093BC008091BC0084FDFCCF4B
:1013B00008958093BB0084E88093BC008091BC00BA
:1013C00087FFFCCF9091B900987F81E0983209F4B3
:1013D00080E0089584E88093BC008091BC0087FF82
:1013E000FCCF8091BB00089580910001811115C050
:1013F00080E40E94AF098093000181110CC082E15A
:101400000E94D90980930001811105C08FEF0E94CD
:10141000D909809300010E94D10984B1807F84B9E9
:1014200085B1807F85B98AB1837F8AB98BB1837F8B
:101430008BB93E98469808950E945A0980930001FE
:101440000E94F40980B38C7080BB81B3836F81BB31
:10145000ECE4F1E0AEE3B1E011921D9281E0EA35F7
:10146000F807D1F78DE399E0892B11F00C943D0931
:1014700008957F928F929F92AF92BF92CF92DF9208
:10148000EF92FF920F931F93CF93DF938091000110
:101490008823E1F080913D018F5F80933D018111B0
:1014A00015C088E994E00E9405080E945A098093BB
:1014B0000001882329F08EE794E00E94050806C009
:1014C0008AE694E00E9405080E94E5088EE3E82E73
:1014D00081E0F82E8701C0E0D0E09924939492E057
:1014E000892EAA24A394B12C3BE5C32E34E0D32E3D
:1014F000C730D10500F580910001811164C080E4FE
:101500000E94AF0980930001811112C082E10E9404
:10151000D9098093000181110BC0C5010C2E01C0B7
:10152000880F0A94EAF780950E94D90980930001F8
:101530000E94D10948C0CA30A1F028F4C83059F03F
:10154000C93061F005C0CC3089F070F0CD3089F041
:10155000209A289810C0219A29980DC0229A2A987A
:101560000AC0239A2B9807C0529A01C0539A5B98DD
:1015700002C03E9A4698E0EAEA95F1F78FB1817091
:101580008925799902C032E001C030E0832B7C9933
:1015900002C034E001C030E0832B7D9902C028E016
:1015A00001C020E0822B7E9902C090E101C090E052
:1015B000892B9FB19095991F9927991F9295990F03
:1015C000907E892B10C080910001811175C080E44C
:1015D0000E94AF0980930001882309F45AC0712C3E
:1015E0000E94D109872DD8019C91981739F18C93CD
:1015F00080910101882301F18091D70180FF04C00F
:1016000080E694E00E9405088091D70180FF0CC01D
:10161000809101011F928F93DF92CF920E949E08CA
:101620000F900F900F900F908091D70180FF04C012
:1016300089E594E00E940508809201010E94F40966
:1016400021960F5F1F4FCE30D10509F051CF809109
:1016500001018823B9F0815080930101882339F07A
:10166000EFE9FFE03197F1F700C000000BC0ECE4B8
:10167000F1E0D7018D917D018193BCE4EB16B1E0DF
:10168000FB06B9F78CED98E0892BC1F00E94DC08CD
:1016900015C083E10E94D9098093000181119FCF79
:1016A00081E40E94AF0980930001811198CF0E94CC
:1016B000EA09782E709494CF80E095CF81E0DF9195
:1016C000CF911F910F91FF90EF90DF90CF90BF903F
:1016D000AF909F908F907F900895E82FF0E0E45BAB
:1016E000FE4F80810895CF92DF92EF92FF920F9389
:1016F0001F93CF93DF9382E494E00E9405088CE46B
:10170000E82E81E0F82EC0E0D0E09DE3C92E94E001
:10171000D92E04E314E0DF93CF93DF92CF920E949F
:101720009E088AE394E00E940508F70181917F01F9
:1017300090E00E9470229F938F931F930F930E94BB
:101740009E0882E394E00E94050821968DB79EB71B
:1017500008960FB6F8949EBF0FBE8DBFCE30D10550
:10176000D1F6DF91CF911F910F91FF90EF90DF9015
:10177000CF9008958B3B910580F4883A910548F508
:10178000853A9105D8F48430910508F0B2C00197EC
:1017900009F06EC081E090E00895803E910508F464
:1017A00067C0883E910508F4A4C09C01205F310900
:1017B0002031310508F05CC090650895853A9105A7
:1017C00009F459C0863A910509F058C082E890E4BE
:1017D0000895883A910509F454C0893A910509F4AD
:1017E00053C08A3A910509F452C08B3A910509F425
:1017F00051C08C3A910509F450C08D3A910509F415
:101800004FC0803B910509F44EC08E3A910509F412
:101810004DC08F3A910509F44CC0813B910509F404
:101820004BC0823B910509F44AC0833B910509F402
:1018300049C0843B910509F448C0853B910509F4F2
:1018400047C0863B910509F446C0873B910509F4E2
:1018500045C0883B910509F444C0893B910509F4D2
:1018600043C08A3B910509F442C080E094E40895A6
:1018700080E090E0089581E890E4089583E890E4A2
:10188000089582EE94E4089589EE94E408958AEE32
:1018900094E4089585EB94E4089586EB94E4089528
:1018A00087EB94E408958CEC94E408958DEC94E433
:1018B000089583E895E408958AE895E4089582E917
:1018C00095E4089584E995E4089581E296E4089505
:1018D00083E296E4089584E296E4089585E296E42E
:1018E000089586E296E4089587E296E408958AE2F0
:1018F00096E4089524E5829FC0011124FC0126E0AE
:10190000729FE00DF11D1124E60FF11DEE0FFF1F78
:10191000E651FF4F859194910895880F991FFC011E
:10192000E05AF040859194910895880F991FFC0129
:10193000E052FF4F85919491089524E5829FC00164
:101940001124FC0146E0749FE00DF11D1124E60F07
:10195000F11DEE0FFF1FE651FF4F859194919C0101
:101960003A9521154FE1340708F429C13F5121155B
:10197000304120F49F700E94950C08959C013053D3
:101980002115304118F49927906C0895811520E5B0
:10199000920769F40E94D81B4FEF84E39CE041500A
:1019A00080409040E1F700C000000C943223813069
:1019B00020E5920751F482EB94E00E9405088091A3
:1019C000D70181608093D70108959C01305521157E
:1019D000304108F05CC0292F33272F703327213086
:1019E0003105E9F4AC0164E0440F551F6A95E1F755
:1019F00044275370BC016370772702C0220F331F46
:101A00006A95E2F73C68242B352B73E0880F991F09
:101A10007A95E1F780769927822B932B08952230CF
:101A2000310529F4982F8827816F906A0895233013
:101A30003105A1F4AC0133E0440F551F3A95E1F7AD
:101A4000407E57708370992721E030E002C0220F5A
:101A5000331F8A95E2F7C9019C6816C0243031050E
:101A600031F5AC0123E0440F551F2A95E1F7407E84
:101A700057708370992721E030E002C0220F331F96
:101A80008A95E2F7C9019A68842B952B08959C01E9
:101A900030572115304118F49F70906208959C01D1
:101AA00030582115304118F49F70906A0895803E97
:101AB0009105E0F4803C910558F58133910509F4D6
:101AC0006FC048F48932910509F463C08A329105E8
:101AD00009F46DC072C089339105E9F0823891052F
:101AE000D1F08533910509F44DC067C0833E91055F
:101AF00081F138F4803E9105B9F0823E9105D9F02C
:101B00005CC0863E910561F1873E9105A1F155C00B
:101B10000E948D0C08952091E90120FD02C021FF53
:101B20004CC080EE90E049C08091E90180FFF9CF80
:101B300089E390E042C08091E90182FF0EC080916C
:101B4000E90184FF03C080E090E037C083EE90E0BD
:101B500034C08091E90182FFF2CF82EE90E02DC087
:101B60008091E90183FF0BC08091E90184FDEBCFF7
:101B700087EE90E022C08091E90183FFF5CF86EEE9
:101B800090E01BC08091E90185FF07C089E290E0E9
:101B900014C08091E90185FFF9CF85E390E00DC085
:101BA0008091E90186FF07C08AE290E006C080913B
:101BB000E90186FFF9CF81E390E00E94BA0B089516
:101BC0000895009739F08A30910514F44D960895E0
:101BD0000697089587E290E008951F93CF93DF93CF
:101BE000FC018281882309F440C0C62FD0E0D42BA9
:101BF00082EE0E9497178D2F82958F7090E00E9441
:101C0000E10D182F0E949717812F0E945F18CE01B7
:101C100088279F70892F90E00E94E10D182F0E9465
:101C20009717812F0E945F18CE01807F992724E0AB
:101C3000969587952A95E1F70E94E10D182F0E944D
:101C40009717812F0E945F18CE018F7099270E94ED
:101C5000E10DC82F0E9497178C2F0E945F1882EE0B
:101C6000DF91CF911F910C945F18DF91CF911F915D
:101C7000089580916D0108959FB7F89410925C01CA
:101C80009FBF9091EF01943009F057C09091E90007
:101C90009F703091EC00232F217030FD20E8922BB3
:101CA00024E02093E9002091EB0020FF43C0209125
:101CB000EE0027FF3FC020915A01222321F02091FE
:101CC000E80025FF37C010925A0126E03091E80065
:101CD00035FD15C03091EF01343061F53091EB00E6
:101CE00035FD28C0215021F481E080935A0122C0A3
:101CF000EFE9FFE03197F1F700C00000E7CF8093F4
:101D0000F1008091E80085FD0AC08091E80080FF25
:101D1000FCCF8091E8008E778093E80006C08FB7F3
:101D2000F89421E020935C018FBF9F709093E900AD
:101D300080E008959F709093E9008FEF0895CF930E
:101D4000DF9300D01F92CDB7DEB79C018091EF01E9
:101D5000843019F593E099833B832A839093E900BB
:101D60008FEF9091E800815095FD06C095ED9A9512
:101D7000F1F700008111F5CF8091E80085FF0DC0DB
:101D800040E050E063E070E0CE0101960E947211E5
:101D90008091E8008E778093E8000F900F900F906D
:101DA000DF91CF910895CF93DF9300D01F92CDB7ED
:101DB000DEB72091EF01243021F522E029839B83B7
:101DC0008A8383E08093E9008FEF9091E80081504F
:101DD00095FD06C095ED9A95F1F700008111F5CFBC
:101DE0008091E80085FF0DC040E050E063E070E0C6
:101DF000CE0101960E9472118091E8008E77809347
:101E0000E8000F900F900F90DF91CF9108959C0103
:101E10008091EF018430F9F482E08093E9009FEF34
:101E20008091E800915085FD06C085ED8A95F1F717
:101E300000009111F5CF8091E80085FF0CC040E0D3
:101E400050E065E070E0C9010E9472118091E800E5
:101E50008E778093E8000895CF93DF93EC01809113
:101E6000EF01843009F047C080910C018823E1F034
:101E700080910D018823C1F085E08093E9008FEF08
:101E80009091E800815095FD06C095E19A95F1F793
:101E900000008111F5CF8091E80085FF2CC040E063
:101EA00050E060E170E017C081E08093E9008FEFBF
:101EB0009091E800815095FD06C095ED9A95F1F757
:101EC00000008111F5CF8091E80085FF14C040E04B
:101ED00050E068E070E0CE010E9472118091E8004D
:101EE0008E778093E80080E1FE01ADE5B1E00190DE
:101EF0000D928A95E1F7DF91CF91089589EE94E0F4
:101F00000E9405088091EE01811109C00E9403130F
:101F10000E9460138091E20084608093E200089543
:101F200085EE94E00E9405081092EE01089581EE7E
:101F300094E00C9405088DED94E00E9405080C9443
:101F4000012D89ED94E00E9405080E94C8220E949C
:101F5000072D0E940A160C94E00D20915B012F5F63
:101F6000822F62E30E94842E992319F020935B0153
:101F7000089510925B0180915C01882371F180913A
:101F8000EF01843041F58091E9008F702091EC00E1
:101F9000922F917020FD90E8892B94E09093E900B6
:101FA0009091EB0090FF14C09091EE0097FF10C04D
:101FB0009091E80095FF03C01092F100F9CF909145
:101FC000E80090FF05C09091E8009E779093E800AC
:101FD0008F708093E90010925C01089542E061ECFB
:101FE00081E00E947C1242E061EC82E00E947C125F
:101FF00042E061EC83E00E947C1242E261EC84E00A
:102000000E947C1242E161EC85E00C947C1280918C
:10201000F101833009F455C030F4813071F0823021
:1020200009F48EC008958A3009F47AC08B3009F41F
:1020300060C0893009F09CC020C08091F001813AD5
:1020400009F096C08091E800877F8093E800809136
:10205000F4019091F501892B21F460E18DE591E087
:1020600003C060E080E090E070E00E94BD118091CC
:10207000E8008B778093E80008958091F001813229
:1020800009F076C08091F4019091F501009719F064
:10209000049709F06DC08091E800877F8093E80085
:1020A0008091E80082FD05C08091EF018111F8CF99
:1020B0005FC08091F10080936D018091E8008B7783
:1020C00053C08091F001813A09F052C08091F4012F
:1020D0009091F501892B09F04BC08091E800877F32
:1020E0008093E8008091E80080FFFCCF80910C0194
:1020F00036C08091F0018132D9F58091F401909140
:10210000F501892BA9F58091E800877F8093E8008D
:102110000E94B1128091F20180930C010C94D81BA3
:102120008091F001813221F58091E800877F8093D2
:10213000E8000E94B1128091F30180936E0108952E
:102140008091F001813AA1F48091E800877F80932B
:10215000E8008091E80080FFFCCF80916E018093C1
:10216000F1008091E8008E778093E8000C94B11222
:10217000089584B7877F84BF0FB6F894A89580919F
:102180006000886180936000109260000FBE90E054
:1021900080E80FB6F89480936100909361000FBEC1
:1021A0000E9496160E9403130E9460138091E20021
:1021B00084608093E2008CE39EE00E940922789480
:1021C0000E94EA150E94981682E091E00E9405168E
:1021D0000E94EF2C88EC94E00E9405088091EF01AA
:1021E000853089F484EC94E00E9405080E948A22DC
:1021F0008091ED01882391F30E94B422882371F32A
:102200000E945C11EBCF0E94C616E8CF292F33271E
:1022100023303105C9F060F42130310581F02230DE
:10222000310509F041C08DE890E021E235E040C081
:1022300021323105E1F02232310531F135C082E140
:1022400090E02EEA35E034C099278130910549F0BD
:1022500028F0029749F5EDEEF4E005C0EDE1F5E078
:1022600002C0E5E0F5E0849190E09F0121C0653077
:10227000D8F4E62FF0E0EE0FFF1FEB5DFE4F20815C
:10228000318189E090E014C0653070F470E0FB01AA
:10229000EE0FFF1FE55EFE4F20813181FB01EA5EFC
:1022A000FE4F808190E004C080E090E020E030E0CC
:1022B000FA0131832083089580E189BD82E189BDDF
:1022C00009B400FEFDCF8091D8008F7D8093D800A7
:1022D0008091E00082608093E0008091E00081FDC9
:1022E000FCCF0895CF92DF92EF92FF920F931F934E
:1022F000CF93DF93EC018B016A010E94D012811110
:1023000033C0C114D10439F0F60180819181081BDA
:10231000190BC80FD91FE12CF12C0115110519F16A
:102320008091E80085FD16C08091E8008E7780934B
:10233000E800C114D10449F0F60180819181E80ED2
:10234000F91EF182E08285E00FC00E94D01288233E
:1023500021F30AC089918093F10001501109FFEF28
:10236000EF1AFF0ADACF80E0DF91CF911F910F9132
:10237000FF90EF90DF90CF9008952091F60130917B
:10238000F7012617370748F06115710539F42091D8
:10239000E8002E772093E80001C0B901FC0120E09D
:1023A0006115710579F18091EF018823F1F1853094
:1023B000F1F18091E80083FD3CC08091E80082FD4E
:1023C0002EC08091E80080FFEBCF2091F300809138
:1023D000F20090E0922B6115710551F08830910563
:1023E00038F421912093F100615071090196F3CFE7
:1023F00021E0089709F020E08091E8008E77809333
:10240000E800CECF2111CFCF0AC08091EF01882301
:1024100061F0853061F08091E80083FD0AC0809111
:10242000E80082FFF2CF80E0089582E0089583E023
:10243000089581E008952091F6013091F701261763
:10244000370748F06115710539F42091E8002E77BF
:102450002093E80001C0B901FC0120E0611571057D
:1024600091F18091EF01882309F440C0853009F48F
:102470003FC08091E80083FD3DC08091E80082FD6F
:102480002FC08091E80080FFE9CF2091F300809178
:10249000F20090E0922B6115710559F0883091059A
:1024A00040F424912093F100319661507109019616
:1024B000F2CF21E0089709F020E08091E8008E77C4
:1024C0008093E800CBCF2111CCCF0AC08091EF01DF
:1024D000882361F0853061F08091E80083FD0AC0B7
:1024E0008091E80082FFF2CF80E0089582E00895B5
:1024F00083E0089581E00895982F973068F59093D0
:10250000E900981739F07091EC002091ED0050919E
:10251000F00003C0242F762F50E021FD02C09F5F02
:10252000ECCF3091EB003E7F3093EB003091ED002B
:102530003D7F3093ED003091EB0031603093EB0044
:102540007093EC002093ED005093F0002091EE008A
:1025500027FDE5CF80E008958F708093E90081E04A
:1025600008958091F00187FF11C08091E80082FDFD
:1025700005C08091EF018111F8CF11C08091E80072
:102580008B770BC08091EF01882349F08091E800A0
:1025900080FFF8CF8091E8008E778093E80008955F
:1025A0002091E4003091E50095E64091EC00842F05
:1025B000817040FF23C08091E80080FD1DC08091A4
:1025C000EF01882399F0853099F08091EB0085FD2B
:1025D00011C04091E4005091E5002417350729F31C
:1025E000915011F09A01E1CF84E0089582E00895BE
:1025F00083E0089581E0089580E008954091E80027
:1026000042FFDDCF08950E9471130E947913E0EE1E
:10261000F0E0808181608083E8EDF0E080818F7759
:10262000808319BCA7EDB0E08C918E7F8C93808164
:102630008F7E80831092EE0108950F931F93CF93A6
:10264000DF930E9471130E947913C8EDD0E0888156
:102650008F77888388818068888388818F7D88834D
:1026600019BC1092EF011092EB011092ED01109243
:10267000EC0100EE10E0F80180818B7F808388817F
:102680008160888342E060E080E00E947C12E1EE9D
:10269000F0E080818E7F8083E2EEF0E080818160D7
:1026A0008083808188608083F80180818E7F808331
:1026B000888180618883DF91CF911F910F91089568
:1026C000E8EDF0E080818F7E8083E7EDF0E08081AF
:1026D0008160808384E082BF81E08093EE010C946E
:1026E0001D13E8EDF0E080818E7F80831092E20080
:1026F00008951092DA001092E10008951F920F924F
:102700000FB60F9211242F933F934F935F936F93C4
:102710007F938F939F93AF93BF93EF93FF9380919A
:10272000E10082FF0BC08091E20082FF07C0809130
:10273000E1008B7F8093E1000E94AD0F8091DA0071
:1027400080FF1FC08091D80080FF1BC08091DA00FD
:102750008E7F8093DA008091D90080FF0DC080E1E8
:1027600089BD82E189BD09B400FEFDCF81E080937F
:10277000EF010E947E0F05C019BC1092EF010E946C
:10278000900F8091E10080FF19C08091E20080FFEE
:1027900015C08091E2008E7F8093E2008091E2007C
:1027A00080618093E2008091D80080628093D8009D
:1027B00019BC85E08093EF010E949B0F8091E1009E
:1027C00084FF30C08091E20084FF2CC080E189BD8D
:1027D00082E189BD09B400FEFDCF8091D8008F7DD4
:1027E0008093D8008091E1008F7E8093E1008091FA
:1027F000E2008F7E8093E2008091E200816080930E
:10280000E2008091EB01882311F084E007C0809101
:10281000E30087FD02C081E001C083E08093EF0107
:102820000E94A10F8091E10083FF29C08091E20006
:1028300083FF25C08091E100877F8093E10082E0E3
:102840008093EF011092EB018091E1008E7F8093E5
:10285000E1008091E2008E7F8093E2008091E200AF
:1028600080618093E20042E060E080E00E947C12A0
:102870008091F00088608093F0000E94970FFF9194
:10288000EF91BF91AF919F918F917F916F915F91E8
:102890004F913F912F910F900FBE0F901F90189561
:1028A0001F920F920FB60F9211242F933F934F93C5
:1028B0005F936F937F938F939F93AF93BF93CF93C8
:1028C000DF93EF93FF93C091E900CF708091EC000C
:1028D000D82FD17080FDD0E81092E9008091F000EF
:1028E000877F8093F00078940E9494141092E900FE
:1028F0008091F00088608093F000CD2BCF70C09362
:10290000E900FF91EF91DF91CF91BF91AF919F913E
:102910008F917F916F915F914F913F912F910F9088
:102920000FBE0F901F9018951F93CF93DF93CDB7D5
:10293000DEB7AA970FB6F894DEBF0FBECDBFE0EFAB
:10294000F1E08091F100819321E0E83FF207C9F7BF
:102950000E9407108091E80083FF24C18091F0015C
:102960009091F101492F50E04A30510508F01AC109
:10297000FA01EA5AFF4F0C94A42E803881F0823875
:1029800009F010C18091F4018F708093E90080916B
:10299000EB0085FB882780F91092E90006C0809142
:1029A000EC019091ED01911182609091E800977F88
:1029B0009093E8008093F1001092F100C8C0282F96
:1029C0002D7F09F0EFC0882319F0823061F0EAC052
:1029D0008091F201813009F0E5C0933009F080E088
:1029E0008093ED012BC08091F201811127C080916D
:1029F000F4018F7009F4D6C08093E9002091EB00B8
:102A000020FF1CC0933021F48091EB00806214C041
:102A10009091EB0090619093EB0021E030E0A901F0
:102A200002C0440F551F8A95E2F74093EA001092C6
:102A3000EA008091EB0088608093EB001092E9003F
:102A40008091E800877F86C08111ACC01091F201AF
:102A50001F778091E3008078812B8093E300809141
:102A6000E800877F8093E8000E94B1128091E8001F
:102A700080FFFCCF8091E30080688093E300111118
:102A800002C082E001C083E08093EF018BC08058D8
:102A9000823008F087C08091F2019091F3018C3D63
:102AA00053E0950779F583E08A838AE289834FB7FB
:102AB000F894DE01139620E03EE051E2E32FF0E0CF
:102AC00050935700E49120FF03C0E295EF703F5F01
:102AD000EF708E2F90E0EA3010F0C79601C0C096DC
:102AE0008D939D932F5F243149F74FBF8091E8006C
:102AF000877F8093E8006AE270E0CE0101960E9431
:102B0000BD1114C0AE014F5F5F4F6091F4010E9490
:102B10000611BC01892B09F445C09091E800977F0C
:102B20009093E80089819A810E941B128091E800AD
:102B30008B778093E80036C08038A1F58091E8005B
:102B4000877F8093E8008091EB018093F100809172
:102B5000E8008E778093E8000E94B11223C08111B3
:102B600021C08091F2019091F30199270297D4F44A
:102B70008091E800877F8093E8008091F201809344
:102B8000EB010E94B1128091EB01811106C080918E
:102B9000E30087FD02C081E001C084E08093EF0183
:102BA0000E94EE0F8091E80083FF0AC08091E80048
:102BB000877F8093E8008091EB0080628093EB0038
:102BC000AA960FB6F894DEBF0FBECDBFDF91CF91AE
:102BD0001F910895CF938091EF018823A1F0C091B8
:102BE000E900CF709091EC00892F817090FD80E812
:102BF000C82B1092E9008091E80083FD0E94941494
:102C0000CF70C093E900CF910895909374018093A1
:102C100073010895E0917301F0917401309721F0F0
:102C20000190F081E02D099480E00895EF92FF92E9
:102C30001F93CF93DF93F82E192FE0917301F0913A
:102C400074013097A9F10280F381E02D09958091FC
:102C5000D70182FF2DC080FF04C083EE96E00E9462
:102C60000508CF2DD12F10E18DEDE82E86E0F82E4E
:102C70008091D70180FF0BC088811F928F93FF92B4
:102C8000EF920E949E080F900F900F900F9011509E
:102C900021961111EDCF8091D70180FF09C08BEDF6
:102CA00096E0DF91CF911F91FF90EF900C94050873
:102CB000DF91CF911F91FF90EF900895E091730104
:102CC000F0917401309721F00480F581E02D099492
:102CD000089520917101309172012817390771F020
:102CE0009093720180937101E0917301F0917401EE
:102CF000309721F00680F781E02D09940895209106
:102D00006F01309170012817390771F090937001AD
:102D100080936F01E0917301F0917401309721F07D
:102D20000084F185E02D0994089508950C9495167A
:102D30000E94CE220E941C0A0C949423CF93C82F89
:102D40008091D70182FF1EC080FF04C08CEF96E007
:102D50000E9405088091D70180FF0CC01F92CF937D
:102D600087EF96E09F938F930E949E080F900F909D
:102D70000F900F908091D70180FF04C085EF96E0FF
:102D80000E9405088C2FCF910C94E00DCF92DF921A
:102D9000EF92FF920F931F93CF93DF93CDB7DEB7E0
:102DA0002B970FB6F894DEBF0FBECDBF0E94390A35
:102DB00086E7C82E81E0D82E00E010E0E02E802FBC
:102DC0000E946D0BF60141916F01F82EF426B1F4CB
:102DD0000F5F1F4F0E30110589F78FEF89838A83AC
:102DE0001B820E94D7228160782F9D838C8349812A
:102DF0005A816B818D810E94691740C09091D701E3
:102E000091FF04C08B870E94730B8B8520E030E01C
:102E10004F2D50E0922FBA01022E02C07595679592
:102E20000A94E2F760FF24C02E83EF8221E030E0B5
:102E3000690102C0CC0CDD1C9A95E2F790E08C2170
:102E40009D21892B09F420E028870E94D7228160E8
:102E5000782F9A8789874E815F8168858A850E944D
:102E60006917F801EA58FE4F8081C826C08206C063
:102E70002F5F3F4F2630310569F6AACF0E94052704
:102E80000E940A16909175018917A1F00E940A16F6
:102E9000809375012B960FB6F894DEBF0FBECDBFA1
:102EA000DF91CF911F910F91FF90EF90DF90CF9026
:102EB0000C949E162B960FB6F894DEBF0FBECDBFB6
:102EC000DF91CF911F910F91FF90EF90DF90CF9006
:102ED0000895CF93DF93CDB7DEB72B970FB6F89455
:102EE000DEBF0FBECDBF4F83588769877A878B8738
:102EF000DE01119686E0FD0111928A95E9F785E0E1
:102F0000FE01379601900D928A95E1F749815A8129
:102F10006B817C818D819E810E946C1E2B960FB6E9
:102F2000F894DEBF0FBECDBFDF91CF910895CF9350
:102F3000C82F882309F4C1C0823859F40E940A16A8
:102F400081FDBBC089E30E9409210E94E32189E33E
:102F50000CC0833879F40E940A1680FDAEC083E568
:102F60000E9409210E94E32183E50E945921CF910B
:102F70000C94E321843859F40E940A1682FD9DC006
:102F800087E40E9409210E94E32187E4EECF8CEFC1
:102F90008C0F813A48F48C2F0E94972B81118DC0A1
:102FA0008C2F0E940921E3CF80E28C0F883048F4F7
:102FB000C77081E001C0880FCA95EAF70E94AC2172
:102FC000D6CF8BE58C0F833078F4C53A29F0C63A1A
:102FD00031F083E890E005C081E890E002C082E82B
:102FE00090E0CF910C94691688E58C0F833108F03E
:102FF00064C0C83A39F1C93A41F1CA3A49F1CB3A09
:1030000051F1CC3A59F1CD3A61F1C03B69F1CE3A78
:1030100071F1CF3A79F1C13B81F1C23B89F1C33BF8
:1030200091F1C43B99F1C53BA1F1C63BA9F1C73B66
:10303000B1F1C83BB9F1C93BC1F1CA3BC9F180E06C
:1030400090E038C082EE90E035C089EE90E032C06A
:103050008AEE90E02FC085EB90E02CC086EB90E0EC
:1030600029C087EB90E026C08CEC90E023C08DEC6B
:1030700090E020C083E891E01DC08AE891E01AC08A
:1030800082E991E017C084E991E014C081E292E006
:1030900011C083E292E00EC084E292E00BC085E2B0
:1030A00092E008C086E292E005C087E292E002C0AA
:1030B0008AE292E0CF910C947F16CF9108958823F5
:1030C00009F44BC0823859F40E940A1681FF45C0AA
:1030D00089E30E9409210E94E32189E30CC083381F
:1030E00071F40E940A1680FF38C083E50E9409210E
:1030F0000E94E32183E50E9459210C94E321843846
:1031000059F40E940A1682FF28C087E40E94092110
:103110000E94E32187E4EFCF9CEF980F913A58F398
:1031200090E2980F983050F4877091E001C0990FA9
:103130008A95EAF7892F0E94B221DFCF9BE5980F8D
:10314000933020F480E090E00C946916885A833123
:1031500020F480E090E00C947F160895882321F0FD
:103160000E94AC210C94E3210895882321F00E9451
:10317000B2210C94E3210895BF92CF92DF92EF9297
:10318000FF920F931F93CF93DF9300D000D000D016
:10319000CDB7DEB77C0185E0F701DE011196019025
:1031A0000D928A95E1F7F70183819481892B09F4C7
:1031B000DDC2908181818F3F19F49F3F09F4D6C20F
:1031C000F7010281258122952F7099838A83898155
:1031D0009A812E830E94C820182FB92E0E94C720E2
:1031E0000E948E1FEB2DE295EF704E2F50E0FA01FA
:1031F000E05AFF4F2E810C94A42E8B2D807F9B2DA7
:103200009F70F92E882319F0F29480EFF8220023A2
:1032100049F0FF2009F457C28F2D0E94BC210E9463
:10322000E32151C2812F0E945F18FF2009F49EC242
:103230008F2D0E94C22126960FB6F894DEBF0FBED6
:10324000CDBFDF91CF911F910F91FF90EF90DF9055
:10325000CF90BF900C94E3213B2D307F8B2D8F704E
:10326000303211F08295807F112319F0113021F155
:103270002CC00023B9F0222309F490C1213009F0B9
:103280008DC126960FB6F894DEBF0FBECDBFDF917D
:10329000CF911F910F91FF90EF90DF90CF90BF9053
:1032A0000C94CC21222319F0213009F45FC28E83C3
:1032B0000E94CF218E8186C1002321F0223008F0A8
:1032C00055C26CC1211152C27DC1002321F02223BD
:1032D00009F464C1F8C1222309F474C109C28B2D19
:1032E00086958695837019F08130D1F03FC2002316
:1032F00021F0812F9B2D937002C080E090E02696F4
:103300000FB6F894DEBF0FBECDBFDF91CF911F91F6
:103310000F91FF90EF90DF90CF90BF900C946916C3
:10332000002321F0812F9B2D937002C080E090E05C
:1033300026960FB6F894DEBF0FBECDBFDF91CF91BA
:103340001F910F91FF90EF90DF90CF90BF900C9462
:103350007F16812F002319F00E948B2502C00E9446
:10336000F32526960FB6F894DEBF0FBECDBFDF91D2
:10337000CF911F910F91FF90EF90DF90CF90BF9072
:103380000C9478268B2D837009F075C00111EEC165
:10339000812F829586958770880F880F912F9F7057
:1033A000C92ED12CE12CF12C082E04C0CC0CDD1C34
:1033B000EE1CFF1C0A94D2F714FF12C00FE010E0BD
:1033C00020E030E004C0000F111F221F331F8A9538
:1033D000D2F7C901B801609570958095909503C0AA
:1033E00060E070E0CB014B2D46954695437042302E
:1033F000C1F060F56C297D298E299F29413051F15A
:1034000026960FB6F894DEBF0FBECDBFDF91CF91E9
:103410001F910F91FF90EF90DF90CF90BF900C9491
:10342000B51F6C297D298E299F2926960FB6F89401
:10343000DEBF0FBECDBFDF91CF911F910F91FF90E7
:10344000EF90DF90CF90BF900C94D11F0E94B51FDA
:10345000C701B60126960FB6F894DEBF0FBECDBFEA
:10346000DF91CF911F910F91FF90EF90DF90CF9060
:10347000BF900C94991F002319F08B2D817001C00F
:103480008695882309F472C1812F8295869587706D
:10349000880F880F912F9F70C92ED12CE12CF12C11
:1034A000082E04C0CC0CDD1CEE1CFF1C0A94D2F7C5
:1034B00014FF12C00FE010E020E030E004C0000F65
:1034C000111F221F331F8A95D2F7C901B8016095D9
:1034D00070958095909503C060E070E0CB014B2D16
:1034E0004695469543704230C1F060F56C297D29C0
:1034F0008E299F29413051F126960FB6F894DEBFF0
:103500000FBECDBFDF91CF911F910F91FF90EF9034
:10351000DF90CF90BF900C948F206C297D298E294D
:103520009F2926960FB6F894DEBF0FBECDBFDF9160
:10353000CF911F910F91FF90EF90DF90CF90BF90B0
:103540000C94AB200E948F20C701B60126960FB6BF
:10355000F894DEBF0FBECDBFDF91CF911F910F91C9
:10356000FF90EF90DF90CF90BF900C947320103FAE
:10357000D1F118F4103E50F4A1C0123F09F463C019
:1035800008F44CC0133F09F473C098C01F708B2D12
:103590008F710023A1F00E940C20812F26960FB678
:1035A000F894DEBF0FBECDBFDF91CF911F910F9179
:1035B000FF90EF90DF90CF90BF900C94AE180E94D8
:1035C0002D20812F26960FB6F894DEBF0FBECDBFFB
:1035D000DF91CF911F910F91FF90EF90DF90CF90EF
:1035E000BF900C94B5180023A9F02111BFC08B2DFA
:1035F0008F7126960FB6F894DEBF0FBECDBFDF9158
:10360000CF911F910F91FF90EF90DF90CF90BF90DF
:103610000C945220223008F0A9C0E9CF0023A9F071
:103620008B2D8F7126960FB6F894DEBF0FBECDBFDF
:10363000DF91CF911F910F91FF90EF90DF90CF908E
:10364000BF900C940C20002359F38B2D8F7126967C
:103650000FB6F894DEBF0FBECDBFDF91CF911F91A3
:103660000F91FF90EF90DF90CF90BF900C942D20A2
:10367000002399F08B2D8F7126960FB6F894DEBF3C
:103680000FBECDBFDF91CF911F910F91FF90EF90B3
:10369000DF90CF90BF900C94F71F26960FB6F8944A
:1036A000DEBF0FBECDBFDF91CF911F910F91FF9075
:1036B000EF90DF90CF90BF900C94ED1F0023A9F006
:1036C000222309F4ADCF812F26960FB6F894DEBFE2
:1036D0000FBECDBFDF91CF911F910F91FF90EF9063
:1036E000DF90CF90BF900C949717222309F4ADCFB1
:1036F000812F26960FB6F894DEBF0FBECDBFDF91A7
:10370000CF911F910F91FF90EF90DF90CF90BF90DE
:103710000C945F184B2D4F70612FC7010E94A708B2
:1037200026960FB6F894DEBF0FBECDBFDF91CF91C6
:103730001F910F91FF90EF90DF90CF90BF900C946E
:10374000111F4B2D4F70612FC70126960FB6F894AD
:10375000DEBF0FBECDBFDF91CF911F910F91FF90C4
:10376000EF90DF90CF90BF900C94ED0D26960FB6A2
:10377000F894DEBF0FBECDBFDF91CF911F910F91A7
:10378000FF90EF90DF90CF90BF9008950E94C921E5
:103790000E949E210E94E3210E94AA270E9478266F
:1037A00080E090E00E94691680E090E00C947F1623
:1037B0000E94B9210C94C61B0E94C820292F229573
:1037C0002F702C3030F42A3048F42250223078F414
:1037D00005C02C3041F02F3031F009C0803E48F058
:1037E000803F29F406C093FB882780F9089580E084
:1037F000089581E00895CF93DF9300D000D01F9209
:10380000CDB7DEB70F900F900F900F900F90DF9114
:10381000CF910895CF93DF9300D000D000D0CDB7E3
:10382000DEB726960FB6F894DEBF0FBECDBFDF9190
:10383000CF9108951F93CF93DF93C091840116E039
:1038400080918501C81799F0D0E01C9FF0011D9F61
:10385000F00D1124EA57FE4F40815181628173813E
:10386000848195810E940A1C2196C770E9CFDF915F
:10387000CF911F9108954091B6015091B701609189
:10388000B8017091B9018091BA019091BB010C947B
:103890000A1C8091BB0182958F7009F054C0809101
:1038A000B801882309F44FC080918401A09185015B
:1038B0004091B9015091BA016091B6017091B70180
:1038C000B6E08A1709F43FC090E041155105C1F1F7
:1038D0007F3F11F46F3FA1F1B89FF001B99FF00D48
:1038E0001124EA57FE4F218127132AC02081261375
:1038F00027C02281211124C0238134812417350758
:1039000010F421503109241B350B283C3105C0F43B
:103910002091BB012F7020612093BB0126E0289FDE
:10392000F001299FF00D1124E557FE4F80818F7023
:103930008061808386EB91E00E94BC180C941A1C75
:1039400001968770BECF0895CF92DF92EF92FF92DB
:103950000F931F93CF93DF93CDB7DEB762970FB668
:10396000F894DEBF0FBECDBF8C0185E0F801DE010B
:103970001D9601900D928A95E1F7D8014C91119610
:103980005C91119712966C918091B9019091BA0156
:10399000009709F475C13091B6017091B7017F3F6E
:1039A00019F43F3F09F46CC1F801C380D480E09062
:1039B000B801EE2009F4BEC02091BB01C816D9069B
:1039C00028F0D601A81BB90BCD0104C080959095B5
:1039D0008C0D9D1DFF24F394883C910578F0F12C0B
:1039E000207F09F0C4C07C2DD98AC88A89890E94A9
:1039F000FB1B86EB91E00E94BC18AFC0822F807F3A
:103A000009F045C0571313C0431311C061110FC013
:103A10002F7020612093BB010E943B1C86EB91E03C
:103A20000E94BC188091BB01F80185832EC0CD286F
:103A300019F15F3F11F44F3FF9F0F62E61111CC0F0
:103A4000809184012091850136E0821709F45BC0E2
:103A500090E0389FF001399FF00D1124EA57FE4F96
:103A60007181571306C07081471303C072817111B1
:103A700003C001968770E9CFF62E662309F41CC1B6
:103A80008091BB0181608093BB01F12C15C157135C
:103A900009C0431307C0611105C08091BB01F80143
:103AA0008583C8C04D875E878D859E856A8B0E9401
:103AB000DC1B6A898823D1F16623C1F12091BB0107
:103AC000822F82958F7090E0029774F08091B601FA
:103AD0009091B70198878F831986DB86CA862C87D9
:103AE000CE0107960E94BC1886E0F801A6EBB1E073
:103AF00001900D928A95E1F70E94491C0E943B1C9F
:103B0000FF24F394D9C04D875E878D859E850E94E2
:103B1000C820292F22952F70223008F0C1C09F7035
:103B200009F0BBC0805E883008F4C6C0C8010E949E
:103B3000BC18E6CFC816D90608F453C0F601E81B36
:103B4000F90BCF01883C910508F450C0F12C7C2D75
:103B5000D98AC88A89890E94FB1BE6EBF1E086E0DE
:103B6000DF011D928A95E9F70E943B1CA5C05713FF
:103B700014C0431312C0611110C08091BB01F80141
:103B80008583C8010E94BC1886E0E6EBF1E0DF0106
:103B90001D928A95E9F7FE2C8FC04D875E878D8533
:103BA0009E856A8B0E94DC1B6A89882309F4BECF3C
:103BB000662309F4BBCF2091BB01822F82958F70C1
:103BC00090E002970CF490CF8091B6019091B701EC
:103BD0009A8389831B82DD82CC822E83CE0101965B
:103BE00081CF809590958C0D9D1DACCFF62E6623D0
:103BF00009F49CCF571333C0431331C02091BB014C
:103C000020FD24C0822F82958F70482F50E04115EF
:103C10005105E1F0D80115962C9315974F305105B9
:103C200049F08F5F982F9295907F822F8F70892B0C
:103C300015968C93C8010E94BC1886E0F801A6EB8B
:103C4000B1E001900D928A95E1F78ECF86E0F80100
:103C5000A6EBB1E001900D928A95E1F72DC04D875A
:103C60005E878D859E850E94DC1B81113DCF8091F2
:103C7000BB0181608093BB01C8010E94BC181CC0BD
:103C8000662309F453CF4D875E878D859E850E94FC
:103C9000DC1B882309F44ACF27CF811143CF0CC006
:103CA000243008F043CF9F7009F43CCFD80115961B
:103CB0009C91907F09F036CF8F2D62960FB6F894C5
:103CC000DEBF0FBECDBFDF91CF911F910F91FF904F
:103CD000EF90DF90CF9008951F93CF93DF93CDB7F0
:103CE000DEB72C970FB6F894DEBF0FBECDBF4F8363
:103CF000588769877A878B879C87CE0107960E94B1
:103D0000A41C882371F08A859B85892B09F441C006
:103D100088858F3F09F065C08F818F3F09F061C0B2
:103D200038C086E0FE013796DE01119601900D92B3
:103D30008A95E1F76A857B856115710551F1FF81EF
:103D4000E885EF3F11F4FF3F21F12091850130E03C
:103D5000C9010196877099274091840150E084172A
:103D6000950709F447C0F983EA837D836C8396E065
:103D7000929FD001939FB00D1124AA57BE4FFE0110
:103D8000319601900D929A95E1F7809385010E94FA
:103D90001A1C16E080918401909185018917B9F170
:103DA000189FC00111248A579E4F0E94A41C88238B
:103DB00071F1E09184011E9FF0011124EA57FE4F3A
:103DC0004081518162817381848195810E940A1CA6
:103DD0008091840190E001968770992780938401F7
:103DE000D9CF4F81588569857A858B859C850E94BE
:103DF0000A1CCFCF0E94D81B10928501109284011B
:103E0000E6EBF1E086E0DF011D928A95E9F72C965A
:103E10000FB6F894DEBF0FBECDBFDF91CF911F91DB
:103E20000895EF92FF920F931F93CF93DF938C012E
:103E3000892B09F46CC0F12CEE24E394E80121965F
:103E4000F8018491843740F4843008F051C0813007
:103E500081F0823019F15BC0853709F444C0A8F1C4
:103E60009CE7980F903708F052C08F770E945F1838
:103E700041C00E5F1F4FFE01849190E2980F983071
:103E800050F48770FE2D01C0FF0F8A95EAF78F2F3F
:103E90000E94BC2114C00E9497172DC00E5F1F4FB7
:103EA000FE01849190E2980F983060F48770FE2DA7
:103EB00001C0FF0F8A95EAF78F2F0E94C2210E944E
:103EC000E32119C00E945F1816C00E5F1F4FFE014C
:103ED000C491CC2381F08FE99FE00197F1F700C0F6
:103EE0000000C150F6CF0E5F1F4FFE01F49003C0DB
:103EF0000E9497178E018F2D882309F49FCFEFE939
:103F0000FFE03197F1F700C000008150F5CFDF915D
:103F1000CF911F910F91FF90EF90089508956093B6
:103F2000C0017093C1018093C2019093C3010C94AE
:103F3000C61B0F931F930091C0011091C1012091E6
:103F4000C2013091C301DC01CB01802B912BA22B4C
:103F5000B32B8093C0019093C101A093C201B09391
:103F6000C3011F910F910C94C61B0F931F930091D7
:103F7000C0011091C1012091C2013091C301DC0147
:103F8000CB0180239123A223B3238093C00190937C
:103F9000C101A093C201B093C3011F910F910C9472
:103FA000C61B0F931F930091C0011091C101209176
:103FB000C2013091C301DC01CB0180279127A227E8
:103FC000B3278093C0019093C101A093C201B09325
:103FD000C3011F910F910C94C61B1092BC0110924B
:103FE000BD011092BE011092BF010C94C61B41E0AE
:103FF00050E060E070E004C0440F551F661F771F5B
:104000008A95D2F74093BC015093BD016093BE01E5
:104010007093BF010C94C61B41E050E060E070E07B
:1040200004C0440F551F661F771F8A95D2F78091F1
:10403000BC019091BD01A091BE01B091BF01482B80
:10404000592B6A2B7B2B4093BC015093BD0160938D
:10405000BE017093BF010C94C61B41E050E060E0CC
:1040600070E004C0440F551F661F771F8A95D2F772
:1040700040955095609570958091BC019091BD01DF
:10408000A091BE01B091BF01482359236A237B232D
:104090004093BC015093BD016093BE017093BF017A
:1040A0000C94C61B41E050E060E070E004C0440F97
:1040B000551F661F771F8A95D2F78091BC0190919A
:1040C000BD01A091BE01B091BF01482759276A27C1
:1040D0007B274093BC015093BD016093BE01709358
:1040E000BF010C94C61B0F931F930091BC0110914C
:1040F000BD012091BE013091BF01DC01CB01802BBD
:10410000912BA22BB32B8093BC019093BD01A09364
:10411000BE01B093BF011F910F910C94C61B0F936A
:104120001F930091BC011091BD012091BE013091FF
:10413000BF01DC01CB0180239123A223B323809311
:10414000BC019093BD01A093BE01B093BF011F912C
:104150000F910C94C61B0F931F930091BC011091FB
:10416000BD012091BE013091BF01DC01CB01802750
:104170009127A227B3278093BC019093BD01A09300
:10418000BE01B093BF011F910F910C94C61B0895FF
:10419000CF92DF92EF92FF920F931F93CF93DF9313
:1041A0008C01C090BC01D090BD01E090BE01F090A8
:1041B000BF018091C0019091C101A091C201B09155
:1041C000C301C82AD92AEA2AFB2ACFE1D0E0D701C5
:1041D000C6010C2E04C0B695A795979587950A94AD
:1041E000D2F780FF07C0B8018C2F0E949D0C813050
:1041F000910531F4219758F7B80180E00E949D0C99
:10420000DF91CF911F910F91FF90EF90DF90CF90B2
:10421000089590910C01992379F190910D019923C2
:1042200059F1982F9695969596959F30A0F4E09128
:104230000E01F0910F01E90FF11D877021E030E0D0
:10424000A90102C0440F551F8A95E2F7CA01918166
:10425000892B818308959091D70190FF29C01F92E7
:104260008F938DE297E09F938F930E949E080F900B
:104270000F900F900F90089520910E0130910F0133
:10428000F90132969FEF40E05191851789F09F3FE9
:1042900019F4511101C0942F4F5F4E30A9F79F3F81
:1042A00039F0F901E90FF11D97FDFA958283089520
:1042B000089590910C01992381F190910D0199231A
:1042C00061F1982F9695969596959F30A8F4E09178
:1042D0000E01F0910F01E90FF11D877021E030E030
:1042E000A90102C0440F551F8A95E2F7CA018095C3
:1042F00091818923818308959091D70190FF1DC0FA
:104300001F928F938FE097E09F938F930E949E0858
:104310000F900F900F900F90089520910E01309103
:104320000F01F9013296205F3F4F9081891301C040
:1043300010823196E217F307C1F7089581E090E00B
:10434000E0910E01F0910F01E80FF91F1082019624
:1043500080319105A9F708959091D601892B80931A
:10436000D601089580959091D60189238093D60136
:1043700008951092D60108959091D501892B8093CC
:10438000D501089580959091D50189238093D50119
:1043900008951092D50108958093C4010895109254
:1043A000C401089580910E0190910F01FC01319696
:1043B0009C01205F3F4F80E0919191118F5FE21748
:1043C000F307D1F70895E0910E01F0910F0180916C
:1043D000D6018083E0910E01F0910F0190818091D0
:1043E000D501892B80838091C401882361F0E091FD
:1043F0000E01F0910F019081892B80830E94D221C0
:1044000081111092C40180910E0190910F010C94C2
:10441000161690933B0180933A010895CF92DF9254
:10442000EF92FF926C01EE24FF24C114D104E10449
:10443000F10421F0C701B60120E101C020E0C72E40
:10444000D82EE92EFF24C114D104E104F10419F09F
:10445000285FC701B6016B017C0154E0F694E79434
:10446000D794C7945A95D1F7C114D104E104F1044B
:1044700019F02C5FC701B6016B017C0142E0F69494
:10448000E794D794C7944A95D1F7C114D104E104B5
:10449000F10419F02E5FC701B601DC01CB01B6951E
:1044A000A79597958795892B8A2B8B2B09F02F5FE2
:1044B000822FFF90EF90DF90CF9008958295982FF4
:1044C000937344E0949F900111248C7C869586958B
:1044D000282B822F8575880F2A7A2695822B08959E
:1044E0001F93CF93DF931F92CDB7DEB799830E94BE
:1044F0005E22182F9981892F0E945E22212F30E0A1
:10450000322F2227A901482BCA010F90DF91CF91AA
:104510001F9108958091EF01843011F120E488E12A
:1045200090E00FB6F894A895809360000FBE20939A
:10453000600083B7817F846083BF83B7816083BF5E
:104540007894889583B78E7F83BF0FB6F894A8952B
:1045500080916000886180936000109260000FBEBF
:10456000089508950C94B122CF930E94B2220E9424
:10457000390A0E94B122C0E08C2F0E946D0B81117C
:1045800004C0CF5FCE30C1F701C081E0CF91089564
:104590000E94D81B0E940A160C94E00D82E084BD94
:1045A00093E095BD9AEF97BD80936E0008952FB765
:1045B000F8948091D8019091D901A091DA01B0913D
:1045C000DB012FBF0895CF92DF92EF92FF920F93FE
:1045D0001F932FB7F8944091D8015091D901609161
:1045E000DA017091DB012FBF6A017B01EE24FF2409
:1045F0008C0120E030E0C016D106E206F30610F48C
:10460000415051099A01281B390BC9011F910F9183
:10461000FF90EF90DF90CF9008951F920F920FB60A
:104620000F9211248F939F93AF93BF938091D801E2
:104630009091D901A091DA01B091DB010196A11D01
:10464000B11D8093D8019093D901A093DA01B09362
:10465000DB01BF91AF919F918F910F900FBE0F9093
:104660001F9018950E940313F8942FEF87EA91E6A4
:10467000215080409040E1F700C0000087E090EBBF
:10468000DC018093F8019093F901A093FA01B093B3
:10469000FB019CE088E10FB6F894A8958093600038
:1046A0000FBE90936000FFCFEF92FF920F931F9386
:1046B000CF93DF93D82FC0E08C2F0E946D0B00E0CA
:1046C00010E0E82EF12CC701002E02C095958795C9
:1046D0000A94E2F780FD06C00F5F1F4F06301105F8
:1046E00091F709C0602F7C2F80E00E947A0C8D1317
:1046F000F3CF81E004C0CF5FCE30F1F680E0DF91F0
:10470000CF911F910F91FF90EF900895CF93C82FF5
:104710008CE20E945423882321F08C2FCF910C949B
:10472000542380E0CF910895CF930E94E324811118
:1047300002C00E94C92482E597E00E940508C5E6F0
:10474000C15049F00E94390A8FE39CE90197F1F7C3
:1047500000C00000F5CF8BE497E00E94050889E2D5
:104760000E948623811113C18AE20E94862381114F
:104770000E94C92485E00E94862381110E94322371
:104780000E94EE248093D70187E00E94862388232D
:10479000A9F18BE10E948623882351F08091D701F3
:1047A00081FB222720F991E0922790FB81F90EC02E
:1047B0008EE00E948623882361F08091D70182FBDE
:1047C000222720F991E0922790FB82F98093D7016C
:1047D00015C080E10E9486239091D701882341F083
:1047E00093FB222720F981E0822780FB93F904C004
:1047F000892F809580FB90F99093D7018091D70104
:104800000E94F2240E9400258093E90180EE0E941C
:104810008623882341F08091E901982F909590FBA1
:1048200080F98093E90189E30E948623882359F067
:104830008091E90181FB222720F991E0922790FBEA
:1048400081F98093E90182EE0E948623882359F042
:104850008091E90182FB222720F991E0922790FBC9
:1048600082F98093E90186EE0E948623882359F01D
:104870008091E90183FB222720F991E0922790FBA8
:1048800083F98093E90183EE0E948623882359F0FF
:104890008091E90184FB222720F991E0922790FB87
:1048A00084F98093E90185E30E948623882359F0E7
:1048B0008091E90185FB222720F991E0922790FB66
:1048C00085F98093E90181E30E948623882359F0CA
:1048D0008091E90186FB222720F991E0922790FB45
:1048E00086F98093E90181E10E948623882359F0AB
:1048F0008091E90187FB222720F991E0922790FB24
:1049000087F98093E9018091E9010E940425809153
:10491000E90187FB882780F980930D0187E20E94D7
:104920008623C82F8EE10E9486238111C2608FE109
:104930000E9486238111C46080E20E948623811137
:10494000C86081E20E9486238111C06182E20E94D8
:1049500086238111C06283E20E9486238111C06494
:1049600084E20E948623882311F0C06802C0CC2311
:1049700029F08C2F0E94FB246C2F03C00E94F72487
:10498000682F70E080E090E0CF910C948F1FCF9162
:1049900008956DEE7EEF80E090E00E94DA2E60E0F8
:1049A00082E090E00E94CC2E60E083E090E00E94E4
:1049B000CC2E60E084E090E00E94CC2E60E085E0A8
:1049C00090E00C94CC2E80E090E00E94C62E21E076
:1049D0008D3E9E4F09F020E0822F089582E090E006
:1049E0000C94BE2E682F82E090E00C94CC2E83E0D5
:1049F00090E00C94BE2E682F83E090E00C94CC2EB7
:104A000084E090E00C94BE2E682F84E090E00C943B
:104A1000CC2E8091DE0180FF0BC06091130185E0F8
:104A2000689FB001112475956795759567952BC0A2
:104A300081FF09C06091130185E0689FB0011124D6
:104A40007595679520C082FF07C06091130185E0CE
:104A5000689FB001112417C09091DF019923D1F014
:104A600060911201961788F72091130185E0289F25
:104A700090011124929FA001939F500D112470E08A
:104A8000CA010E94902E6038710540F461157105CD
:104A900019F406C065E070E0862F08958FE7089549
:104AA00081E008958091DE0180FF08C060911101CE
:104AB00070E0759567957595679521C081FF06C073
:104AC0006091110170E07595679519C082FF04C06F
:104AD0006091110170E010C09091DF01992399F06D
:104AE000609110019617A0F780911101899FC00174
:104AF000112470E00E94902E6038710540F4611519
:104B0000710519F406C061E070E0862F08958FE703
:104B1000089581E00895803F21F40E940925819540
:104B200004C0813F29F40E9409258093E201089581
:104B3000823F21F40E940925819504C0833F29F416
:104B40000E9409258093E1010895893F19F40E948C
:104B5000522505C08A3F31F40E94522581958093E9
:104B6000E30108958B3F21F40E945225819504C0F2
:104B70008C3F29F40E9452258093E4010895843FDC
:104B800021F48091E001816017C0853F21F480917C
:104B9000E001826011C0863F21F48091E0018460D1
:104BA0000BC0873F21F48091E001886005C0883FF9
:104BB00031F48091E00180618093E00108958D3FA0
:104BC00021F48091DE0181600BC08E3F21F4809141
:104BD000DE01826005C08F3F29F48091DE01846090
:104BE0008093DE010895803F39F48091E20187FFD0
:104BF0006CC01092E20169C0813F29F48091E2010A
:104C00001816BCF362C09091E101823F29F497FF2E
:104C10005CC01092E10159C0833F19F41916CCF31E
:104C200054C0893F41F48091E30118160CF04DC047
:104C30001092E3014AC08A3F29F48091E30187FF83
:104C400044C0F6CF8B3F39F48091E40187FF3DC02B
:104C50001092E4013AC08C3F29F48091E4011816C7
:104C6000BCF333C0843F21F48091E0018E7F17C0F4
:104C7000853F21F48091E0018D7F11C0863F21F4B2
:104C80008091E0018B7F0BC0873F21F48091E00190
:104C9000877F05C0883F31F48091E0018F7E80934B
:104CA000E00113C08D3F21F48091DE018E7F0BC0A7
:104CB0008E3F21F48091DE018D7F05C08F3F29F466
:104CC0008091DE018B7F8093DE018091E101811173
:104CD0000EC08091E20181110AC08091E30181112F
:104CE00006C08091E401811102C01092DF01089595
:104CF0008091D70183FF7EC08EE897E00E9405086F
:104D00008091E0011F928F9389E897E09F938F93A2
:104D10000E949E0887E897E00E9405088091E101C3
:104D2000282F082E000C330B3F938F9384E897E0D5
:104D30009F938F930E949E0882E897E00E94050847
:104D40008091E201282F082E000C330B3F938F93A4
:104D50008FE797E09F938F930E949E088DE797E0DF
:104D60000E9405088091E301282F082E000C330BC8
:104D70003F938F938AE797E09F938F930E949E08BB
:104D800088E797E00E9405088091E401282F082E0B
:104D9000000C330B3F938F9385E797E09F938F939E
:104DA0000E949E0882E797E00E9405088091DF013B
:104DB0001F928F938FE697E09F938F930E949E0898
:104DC0008DE697E00E9405088091DE011F928F9387
:104DD0008AE697E09F938F930E949E0887E697E06C
:104DE0000E9405088DB79EB74C960FB6F8949EBFEB
:104DF0000FBE8DBF80EE91E00E945E160E94D7220A
:104E00009093DD018093DC0108951F93CF93DF938E
:104E10008091DC019091DD010E94E322AC01909130
:104E2000DF01992321F02091140130E006C0209188
:104E300015018AE0289F900111244217530708F4B6
:104E400085C08091E101C091E201D091E301109110
:104E5000E401811107C0C11175C0D11173C01111D6
:104E600071C074C09F3F19F09F5F9093DF011816C7
:104E700024F40E9409258093E1018091E10187FFDC
:104E800005C00E94092581958093E1011C1624F438
:104E90000E9409258093E2018091E20187FF05C00D
:104EA0000E94092581958093E2016091E1016623CA
:104EB00031F1C091E201CC2311F1062E000C770BE9
:104EC000880B990B0E948B2D23E333E343E35FE3CD
:104ED0000E94EF2D0E94532D6093E1016C2FCC0FA7
:104EE000770B880B990B0E948B2D23E333E343E36D
:104EF0005FE30E94EF2D0E94532D6093E2011D1687
:104F000024F40E9452258093E3018091E30187FFFE
:104F100005C00E94522581958093E301111624F467
:104F20000E9452258093E4018091E40187FF05C02F
:104F30000E94522581958093E401DF91CF911F91CA
:104F40000C9478269F3F09F08FCFA0CFDF91CF91AF
:104F50001F910895E0EEF1E085E0DF011D928A9552
:104F6000E9F71092DF011092DE01089581EB99E0DC
:104F70000E9405081F9281E08F931F9285E08F9316
:104F800083E699E09F938F930E949E080F900F9065
:104F90000F900F900F900F9008958330E9F128F44F
:104FA000813061F0823009F10895853009F462C0E2
:104FB00008F449C0863009F474C008958091150141
:104FC000262F30E0280F311D2F3F310524F4680FC4
:104FD0006093150103C08FEF809315018091150137
:104FE0001F928F938CE998E072C080911401262F54
:104FF00030E0280F311D2F3F310524F4680F6093F6
:10500000140103C08FEF80931401809114011F924B
:105010008F938AE898E05BC080911301262F30E0DF
:10502000280F311D2F3F310524F4680F60931301C1
:1050300003C08FEF80931301809113011F928F9310
:1050400087E798E044C080911201262F30E0280FB6
:10505000311D2F3F310524F4680F6093120103C006
:105060008FEF80931201809112011F928F9382E63D
:1050700098E02DC080911101262F30E0280F311DBE
:105080002F3F310524F4680F6093110103C08FEFA7
:1050900080931101809111011F928F9389E498E010
:1050A00016C080911001262F30E0280F311D2F3FB0
:1050B000310524F4680F6093100103C08FEF8093D3
:1050C0001001809110011F928F938EE298E09F93C0
:1050D0008F930E949E080F900F900F900F9008954D
:1050E000833081F128F4813059F08230D1F0089575
:1050F000853009F449C0B8F1863009F456C00895E6
:1051000080911501681720F4861B8093150102C059
:1051100010921501809115011F928F938FE198E0F5
:1051200054C080911401681720F4861B80931401E9
:1051300002C010921401809114011F928F938DE090
:1051400098E043C080911301681720F4861B809378
:10515000130102C010921301809113011F928F93CB
:105160008AEF97E032C080911201681720F4861B05
:105170008093120102C010921201809112011F92BD
:105180008F9385EE97E021C080911101681720F47C
:10519000861B8093110102C01092110180911101B0
:1051A0001F928F938CEC97E010C0809110016817CC
:1051B00020F4861B8093100102C010921001809190
:1051C00010011F928F9381EB97E09F938F930E9422
:1051D0009E080F900F900F900F900895CF93C82FB7
:1051E0001F928F9386EB9AE09F938F930E949E0865
:1051F00081E090E0A0E0B0E0BC01CD0104C0660F0A
:10520000771F881F991FCA95D2F70E948F1F0F9092
:105210000F900F900F90CF910C94D81BCF938D319E
:1052200009F465C0B0F58E3009F4CCC100F58730C3
:1052300009F49BC1A8F4863009F06DC28091D701B2
:10524000817F8E7F8093D7018BEB9AE00E940508C7
:1052500080E09FE00E94050881E08093E60180C124
:10526000883009F44FC08B3009F47CC154C28631B8
:1052700009F4F0C138F4803109F4B8C1813109F47E
:1052800030C249C2893109F4CEC18B3109F486C1DB
:1052900042C2853309F437C248F4873209F433C275
:1052A00008F433C2893209F42EC235C2833438F48B
:1052B0008A3308F02CC2883309F454C12CC28334D9
:1052C00009F421C2883409F026C20E94D81B8FEE4F
:1052D0009EE00E9405089FEF23ED80E3915020405F
:1052E0008040E1F700C000000E94322339C18FE006
:1052F0009FE00E9405080E940D2D0E940A160E9440
:10530000E00D2EC184E09FE00E9405088CEC9CE03B
:105310000E9405080E94F7241F928F9389EC9CE05D
:105320009F938F930E949E0887EC9CE00E94050843
:105330000E94EE24C82F84EB9CE00E9405081F9277
:10534000CF938FEA9CE09F938F930E949E088DEAF3
:105350009CE00E94050883EA9CE00E9405088C2FCF
:1053600081701F928F9380EA9CE09F938F930E949D
:105370009E088EE99CE00E94050884E99CE00E945A
:105380000508C1FB882780F91F928F9381E99CE073
:105390009F938F930E949E088FE89CE00E940508CF
:1053A00083E89CE00E940508C2FB882780F91F92D1
:1053B0008F9380E89CE09F938F930E949E088EE7D6
:1053C0009CE00E94050885E79CE00E940508C3FB5D
:1053D000CC27C0F91F92CF9382E79CE09F938F93D5
:1053E0000E949E0880E79CE00E9405080E9400251C
:1053F000C82F8CE59CE00E9405081F92CF9387E59B
:105400009CE09F938F930E949E0885E59CE00E94FC
:1054100005088CE39CE00E9405088C2F81701F9288
:105420008F9389E39CE09F938F930E949E088DB792
:105430009EB780960FB6F8949EBF0FBE8DBF87E3D0
:105440009CE00E94050880E29CE00E940508C1FBE8
:10545000882780F91F928F938DE19CE09F938F9313
:105460000E949E088BE19CE00E94050889E09CE078
:105470000E940508C2FB882780F91F928F9386E05F
:105480009CE09F938F930E949E0884E09CE00E9482
:10549000050882EF9BE00E940508C3FB882780F97E
:1054A0001F928F938FEE9BE09F938F930E949E0895
:1054B0008DEE9BE00E94050883EE9BE00E940508AC
:1054C000C4FB882780F91F928F9380EE9BE09F9307
:1054D0008F930E949E088EED9BE00E9405088CEC45
:1054E0009BE00E940508C5FB882780F91F928F93D7
:1054F00089EC9BE09F938F930E949E0887EC9BE032
:105500000E9405088BEA9BE00E940508C6FB8827DD
:1055100080F91F928F9388EA9BE09F938F930E945C
:105520009E0886EA9BE00E9405088EE99BE00E94A7
:105530000508C7FBCC27C0F91F92CF938BE99BE0EE
:105540009F938F930E949E0889E99BE00E94050823
:105550008DB79EB74C960FB6F8949EBF0FBE8DBF09
:10556000C1E0DEC082EE9AE05BC08091D701C82F17
:10557000C17080FF09C082EE9EE00E940508809104
:10558000D701817F8E7F47C086ED9EE00E9405088F
:105590008091D70181608093D701E2CF9091D701AC
:1055A00091FBCC27C0F981E0C827892FC0FB81F986
:1055B0008093D701CC2319F089EC9EE027C08BEBB8
:1055C0009EE02EC09091D70192FBCC27C0F981E0DC
:1055D000C827892FC0FB82F98093D701CC2319F00B
:1055E0008CEA9EE013C08CE99EE01AC09091D7012E
:1055F00093FBCC27C0F981E0C827892FC0FB83F932
:105600008093D701CC2351F080E99EE00E940508E9
:105610008091D70181608093D70182C083E89EE0AA
:105620000E9405089DCF84E79EE00E94050888E45B
:105630009EE00E9405088BE09EE00E9405088EED2A
:105640009DE00E9405088AE99DE00E9405088CE61D
:105650009DE0E6CF8EE59DE00E9405080E940A16B7
:105660001F928F9384E49DE09F938F930E949E08E6
:1056700080910C011F928F938DE29DE09F938F93F9
:105680000E949E0880916E011F928F938AE19DE097
:105690009F938F930E949E0880910D011F928F937C
:1056A00087E09DE09F938F930E949E088091D80190
:1056B0009091D901A091DA01B091DB01BF93AF9332
:1056C0009F938F9383EF9CE09F938F930E949E08FC
:1056D0008DB79EB746960FB6F8949EBF0FBE8DBF8E
:1056E0003FCF0E94D81BC0910D0181E0C827C09315
:1056F0000D01CC2329F089EE9CE00E94050810C022
:105700008EED9CE08DCF80E003C08D5101C08953A8
:105710000E94EE2825CF8CED9CE00E940508C0E099
:105720008C2FCF91089580E008950C94932BCF9304
:10573000C82F8091E601813081F020F0823009F499
:105740004FC045C1E0910E01F0910F018081813180
:1057500069F0823209F03DC109C0E0910E01F0917B
:105760000F018081813111F0823261F48C2F0E940F
:10577000952B811104C08C2F0E940E292FC081E02F
:1057800090E02CC08C2F0E94932B811126C0C43135
:10579000E1F070F4CB3081F0C031D1F40E94B62733
:1057A0008EEA9AE00E94050882E08093E60115C027
:1057B000C93259F0C83361F48BEB9AE00E940508B6
:1057C00082EB9AE00E94050808C01092E60103C12E
:1057D0008CEA9AE00E940508FEC081E08170FDC05D
:1057E000C43220F5CE3108F0C0C0CB3099F1C8F4F6
:1057F000C73009F0D2C08AE08093150194E19093FC
:10580000140193E0909313018093120188E0809338
:10581000110188E28093100182E599E00E94050859
:10582000BFC0C33149F1C431C1F0B7C0CB3409F4B2
:10583000A9C028F4C93289F0C83361F0AEC0C135BF
:1058400009F49EC0C23509F499C0CE3409F0A5C050
:105850006AE09EC00E94B627A3C08091E50188231C
:1058600019F01092E5019CC08FE599E00E940508AF
:1058700081E08093E601B1C089E399E00E940508C8
:1058800087E299E00E940508809115011F928F938D
:1058900084E299E09F938F930E949E0882E299E0B0
:1058A0000E94050880E199E00E940508809114019A
:1058B0001F928F938DE099E09F938F930E949E0893
:1058C0008BE099E00E9405088CEF98E00E940508A3
:1058D000809113011F928F9389EF98E09F938F938C
:1058E0000E949E0887EF98E00E94050886EE98E0E7
:1058F0000E940508809112011F928F9383EE98E019
:105900009F938F930E949E0881EE98E00E94050865
:105910008CEC98E00E940508809111011F928F93F2
:1059200089EC98E09F938F930E949E0887EC98E003
:105930000E94050880EB98E00E9405088091100104
:105940001F928F938DEA98E09F938F930E949E08F9
:105950008BEA98E00E9405088DB79EB748960FB66F
:10596000F8949EBF0FBE8DBF1BC0CE51EC2FF0E050
:10597000E15DFE4F80818093E50112C061E003C0CC
:1059800061E006C06AE08091E5010E94CD2708C071
:105990008091E5010E94702803C080E599E013C062
:1059A0008091E501882369F01F928F938AE499E042
:1059B0009F938F930E949E080F900F900F900F90CF
:1059C00004C087E499E00E94050881E006C01092B7
:1059D000E60180E002C080E001CFCF910895E1E8C8
:1059E000F0E08081886080838081816080838FB7D0
:1059F000F89493E09093890090ED909388008FBF86
:105A00000895EFE6F0E08081826080830895EFE6FC
:105A1000F0E080818D7F80830895EFE6F0E0908153
:105A200082E08927808308951F920F920FB60F920C
:105A300011242F933F934F935F936F937F938F9393
:105A40009F93AF93BF93EF93FF938091E701909162
:105A5000E80101969093E8018093E701811103C06A
:105A600082E00E94E00DE091E801E695E695F0E025
:105A7000E15EF04FE4918091E7018E1303C080E076
:105A80000E94E00DFF91EF91BF91AF919F918F9197
:105A90007F916F915F914F913F912F910F900FBE2A
:105AA0000F901F9018950E945A2D6894B1110C9474
:105AB000E92D08950E94CE2D88F09F5798F0B92FB8
:105AC0009927B751B0F0E1F0660F771F881F991F33
:105AD0001AF0BA95C9F714C0B13091F00E94E82DC0
:105AE000B1E008950C94E82D672F782F8827B85FD0
:105AF00039F0B93FCCF3869577956795B395D9F78B
:105B00003EF490958095709561957F4F8F4F9F4F94
:105B10000895E89409C097FB3EF4909580957095A0
:105B200061957F4F8F4F9F4F9923A9F0F92F96E9E9
:105B3000BB279395F695879577956795B795F1115E
:105B4000F8CFFAF4BB0F11F460FF1BC06F5F7F4FFB
:105B50008F4F9F4F16C0882311F096E911C077230D
:105B600021F09EE8872F762F05C0662371F096E816
:105B7000862F70E060E02AF09A95660F771F881FE5
:105B8000DAF7880F9695879597F9089557FD9058FD
:105B9000440F551F59F05F3F71F04795880F97FBF1
:105BA000991F61F09F3F79F08795089512161306AB
:105BB0001406551FF2CF4695F1DF08C016161706DA
:105BC0001806991FF1CF869571056105089408950F
:105BD000E894BB2766277727CB0197F908950E94A1
:105BE000022E0C94732E0E94652E38F00E946C2EAB
:105BF00020F0952311F00C945C2E0C94622E11244D
:105C00000C94E92D0E94C62D70F3959FC1F3950F5A
:105C100050E0551F629FF001729FBB27F00DB11D30
:105C2000639FAA27F00DB11DAA1F649F6627B00DC0
:105C3000A11D661F829F2227B00DA11D621F739FA9
:105C4000B00DA11D621F839FA00D611D221F749FB7
:105C50003327A00D611D231F849F600D211D822FFE
:105C6000762F6A2F11249F5750409AF0F1F0882325
:105C70004AF0EE0FFF1FBB1F661F771F881F915052
:105C80005040A9F79E3F510580F00C945C2E0C9477
:105C9000E92D5F3FE4F3983ED4F3869577956795B9
:105CA000B795F795E7959F5FC1F7FE2B880F911D7C
:105CB0009695879597F9089597F99F6780E870E022
:105CC00060E008959FEF80EC089500240A94161672
:105CD000170618060906089500240A9412161306DA
:105CE000140605060895092E0394000C11F4882368
:105CF00052F0BB0F40F4BF2B11F460FF04C06F5F84
:105D00007F4F8F4F9F4F0895991B79E004C0991FD3
:105D1000961708F0961B881F7A95C9F78095089505
:105D200097FB072E16F4009407D077FD09D00E9448
:105D3000AA2E07FC05D03EF4909581959F4F0895BB
:105D4000709561957F4F0895EE0FFF1F0590F491B8
:105D5000E02D0994AA1BBB1B51E107C0AA1FBB1F62
:105D6000A617B70710F0A61BB70B881F991F5A95E7
:105D7000A9F780959095BC01CD010895F999FECFC2
:105D800092BD81BDF89A992780B50895A8E1B0E049
:105D900042E050E00C94E12E262FF999FECF1FBA75
:105DA00092BD81BD20BD0FB6F894FA9AF99A0FBE44
:105DB000019608950E94CC2E272F0C94CD2EDC0145
:105DC000CB01FC01F999FECF06C0F2BDE1BDF89A06
:105DD000319600B40D9241505040B8F70895F894B0
:025DE000FFCFF3
:105DE2002002390E2C0F070FD30E9F0E0101C501A1
:105DF20028080A03140A3F4D3620399C064F06191B
:105E020006F905C00533054C0565057E059E0501AD
:0A5E1200020304050607080900005A
:00000001FF
